:100000000C944C030C9493030C9493030C9493035F
:100010000C9493030C9493030C9493030C94930308
:100020000C9493030C9493030C94BB0C0C948D0DC3
:100030000C9493030C9493030C9493030C949303E8
:100040000C9493030C94B1210C9493030C9493039C
:100050000C9493030C94431B0C9493030C94930300
:100060000C9493030C9493030C9493030C949303B8
:100070000C9493030C9493030C9493030C949303A8
:100080000C9493030C9493030C9493030C94930398
:100090000C9493030C9493030C9493030C94930388
:1000A0000C9493030C9493030C949303A103A60361
:1000B000AB03B003B503BA03BF03C403C903FA0D0E
:1000C0001C0E0F0F1C0E0F0F610E840E0F0FD90E9A
:1000D000EC0ED611D61105120512481282128F1499
:1000E0008F149B128F149013901363148F148F141A
:1000F0007A14012E022E012C022C0001E10135029E
:100100003502E100013502350001E1012E022E0128
:100110002C022C02E10001E6012E022E02E6012C47
:10012000022C0001E10130023002E1012C022C001E
:1001300001E10164026402E100016402640001E67D
:100140000130023002E6012C022C000000002200E7
:10015000C001C002C003C004C005C006C007C0087B
:10016000C02E002D0237021E020452000025141476
:100170000004001D00F400387426141A0015001B3A
:1001800000F500377124140900160006002B00C189
:1001900000271413001700190036782D0031020AC9
:1001A00000070005000000230201541F0200003672
:1001B0000200003500C5003200000027020000499F
:1001C0000021140D000B000E000000240225020F78
:1001D000001100100050004C002602180008004FCB
:1001E0000029002C00C3001C000C005100C700288F
:1001F00000C4002F001200520020022A001F1434F5
:1002000000330038020252000024160100010001F0
:1002100000010000000100010001000100010001D7
:1002200000010001000100010001003778251601DE
:10023000000100010001000100261601000100017B
:100240000036710100010001000100010000000101
:1002500000010001000000010000002414010064FE
:100260000000000100000001002102010001000166
:100270000000000100010001000100010001000177
:1002800000010001000100010001000100C800019F
:1002900000010001002E140100C90001000100014D
:1002A00000010001003100010001000100035200C3
:1002B0000001000100010001000100000001000137
:1002C000002000010001000100010001001F0001E9
:1002D0000001000100010001001E000100010001F9
:1002E000000100220227002100010001000100019D
:1002F00000010001000000010001000100000001F8
:1003000000000001000100010000000100000001E8
:10031000000100010001004A00000001000100C2CC
:1003200000220026004A0001000100C60023004D03
:1003300000010001000100010024004E0001000145
:10034000000100010025004B000100010001000137
:100350000001000100010000000100010001000196
:100360000001000000010001002000010001000167
:1003700000010001001F0001000100010001000157
:10038000001E0001000100010001002202270021DF
:100390000001000100010001000100010000000156
:1003A0000001000100000001000000010001000147
:1003B0000000000100000001000100010001004AEE
:1003C00000000001000100C200220026004A0001D6
:1003D000000100CA0023004D0001000100010001DE
:1003E0000024004E00010001000100010025004B27
:1003F00000010001000100010001000100010000F6
:1004000000220001000100010001000000010001C4
:10041000003C00010001000100010001003B00015F
:100420000001000100010001003A0001000100018B
:10043000000100010001003D000100010001000178
:1004400000010001000000010001000100000001A6
:100450000000000100010001000000010000000197
:100460000001000100010030140000010001000142
:10047000003E00420001000100010001003F004376
:1004800000010001000100010040004400010001E2
:1004900000010001004100450001000100010001D0
:1004A0000001000100010000001603450072006712
:1004B000006F0044006F007800200045005A0000E3
:1004C0000016034500720067006F0044006F00785B
:1004D00000200045005A0000000403090409026DD1
:1004E00000040100A0FA0904000001030101000951
:1004F0002111010001223F000705810308000A09BC
:100500000401000103010200092111010001224D33
:10051000000705820308000A090402000103000025
:10052000000921110100012236000705830308009C
:100530000A09040300010300000009211101000160
:100540002239000705840310000112011001000088
:100550000008EDFE07130100010200010501090674
:10056000A101050719E029E7150025019508750186
:10057000810205081901290595057501910295016A
:100580007503910105071900297715002501957854
:1005900075018102C005010980A1018502160100D3
:1005A00026B7001A01002AB700751095018100C016
:1005B000050C0901A1018503160100269C021A0100
:1005C000002A9C02751095018100C005010902A155
:1005D000010901A100050919012905150025019549
:1005E0000575018102950175038101050109300935
:1005F000311581257F9502750881060938158125F9
:100600007F950175088106050C0A38021581257F42
:10061000950175088106C0C005010906A1010507FD
:1006200019E029E71500250195087501810295015A
:1006300075088101050819012905950575019102C3
:100640009501750391010507190029FF150025FF84
:10065000950675088100C000000000000000000041
:100660000000010204060A0F17202C3A4A5D718728
:100670009DB3C7DAE9F5FCFFFCF5E9DAC7B39D875E
:10068000715D4A3A2C20170F0A060402010000008F
:10069000000000000000000011241FBECFEFDAE0D0
:1006A000DEBFCDBF04B603FE27C08091ED0190915F
:1006B000EE01A091EF01B091F0018730904BA7407F
:1006C000B04BD1F41092ED011092EE011092EF01B7
:1006D0001092F00114BE84B7877F84BF0FB6F894E0
:1006E000A8958091600088618093600010926000FE
:1006F0000FBEE0E0FFE3099511E0A0E0B1E0E4E027
:10070000F7E402C005900D92A433B107D9F721E0B8
:10071000A4E3B1E001C01D92AD3EB207E1F70E9433
:10072000020A0C9480230C940000FC018281462F65
:1007300050E04930510590F5FA01EA5AFF4F0C9408
:100740003523882359F18EE391E00895882331F110
:1007500089E391E00895882309F180E391E0089509
:100760008823E1F083E291E008958823B9F086E1DF
:1007700091E00895882391F089E091E0089588231D
:1007800069F084E091E00895882341F08BEF90E0D8
:100790000895882319F082EF90E0089580E090E0BA
:1007A000089508950C94D1030C94D10356985E9843
:1007B00025982D9826982E9827982F988FEF90E0BF
:1007C000909389008093880090938B0080938A0097
:1007D00090938D0080938C00259A2D9A2FEF80E7BF
:1007E00092E0215080409040E1F700C00000269A3E
:1007F0002E9A2FEF80E792E0215080409040E1F761
:1008000000C00000279A2F9A2FEF80E792E0215036
:1008100080409040E1F700C0000025982D982FEF10
:1008200080E792E0215080409040E1F700C0000056
:1008300026982E982FEF80E792E02150804090403C
:10084000E1F700C0000027982F9856985E982598E9
:100850002D9826982E9827982F98089589EA8093A6
:10086000800089E08093810024982C983F988AB179
:100870008F748AB96E98479A8BB1806B8BB9769AD0
:100880000E94D6030C94D20380E2809300018091F1
:10089000340181110EC00E94930481E080933401E1
:1008A0002FEF83ED90E3215080409040E1F700C0AE
:1008B000000080E40E9499048093000181112EC001
:1008C0000E94C30480930001811128C00E94C304C8
:1008D00080930001811122C08FE30E94C3048093A2
:1008E000000181111BC00E94BB0480E40E94990496
:1008F00080930001811112C08CE00E94C304809398
:10090000000181110BC00E94C3048093000181117A
:1009100005C08FE30E94C304809300010E94BB04C2
:100920008091000108951092B9008AE08093B80088
:10093000089594EA9093BC009091BC0097FFFCCF7F
:100940009091B900987F983021F0903111F081E0BA
:1009500008958093BB0084E88093BC008091BC0024
:1009600087FFFCCF8091B900887F883111F08034F7
:1009700071F780E0089584E98093BC008091BC0009
:1009800084FDFCCF08958093BB0084E88093BC0075
:100990008091BC0087FFFCCF9091B900987F81E0E7
:1009A000983209F480E0089584E88093BC00809137
:1009B000BC0087FFFCCF8091BB00089580910001AF
:1009C000811115C080E40E94990480930001811177
:1009D0000CC082E10E94C30480930001811105C014
:1009E0008FEF0E94C304809300010E94BB0484B176
:1009F000807F84B985B1807F85B98AB1837F8AB9C8
:100A00008BB1837F8BB93E98469808950E94440429
:100A1000809300010E94DE0480B38C7080BB81B3A0
:100A2000836F81BBE4E4F1E0A6E3B1E011921D9293
:100A300081E0E235F807D1F70C942E049F92AF9233
:100A4000BF92CF92DF92EF92FF920F931F93CF93BB
:100A5000DF9380910001882379F0809135018F5FC9
:100A600080933501811108C00E94440480930001E5
:100A7000811102C00E94D60386E3E82E81E0F82EA1
:100A80008701C0E0D0E0BB24B39492E0A92ECC242F
:100A9000C394D12CC730D10500F58091000181119C
:100AA00064C080E40E94990480930001811112C007
:100AB00082E10E94C3048093000181110BC0C60132
:100AC0000C2E01C0880F0A94EAF780950E94C30497
:100AD000809300010E94BB0448C0CA30A1F028F4F2
:100AE000C83059F0C93061F005C0CC3089F070F0E1
:100AF000CD3089F0209A289810C0219A29980DC0ED
:100B0000229A2A980AC0239A2B9807C0529A01C0A9
:100B1000539A5B9802C03E9A4698E0EAEA95F1F74C
:100B20008FB181708B25799902C032E001C030E02D
:100B3000832B7C9902C034E001C030E0832B7D9987
:100B400002C028E001C020E0822B7E9902C090E123
:100B500001C090E0892B9FB19095991F9927991F0B
:100B60009295990F907E892B0FC080910001811181
:100B70004AC080E40E94990480930001882381F197
:100B8000912C0E94BB04892DD8019C91981719F0D3
:100B90008C93A09201010E94DE0421960F5F1F4FEB
:100BA000CE30D10509F076CF80910101882369F11B
:100BB000815080930101882339F0EFE9FFE03197FC
:100BC000F1F700C0000021C0E4E4F1E0D7018D910D
:100BD0007D018193B4E4EB16B1E0FB06B9F715C0D3
:100BE00083E10E94C304809300018111C9CF81E495
:100BF0000E949904809300018111C2CF0E94D40405
:100C0000982E9094BECF80E0BFCF0E94D40381E0A5
:100C1000DF91CF911F910F91FF90EF90DF90CF90D8
:100C2000BF90AF909F900895E82FF0E0EC5BFE4FEF
:100C30008081089508958B3B910580F4883A910551
:100C400048F5853A9105D8F48430910508F0B2C092
:100C5000019709F06EC081E090E00895803E910513
:100C600008F467C0883E910508F4A4C09C01205F89
:100C700031092031310508F05CC090650895853A4E
:100C8000910509F459C0863A910509F058C082E8E7
:100C900090E40895883A910509F454C0893A910581
:100CA00009F453C08A3A910509F452C08B3A910570
:100CB00009F451C08C3A910509F450C08D3A910560
:100CC00009F44FC0803B910509F44EC08E3A91055E
:100CD00009F44DC08F3A910509F44CC0813B910550
:100CE00009F44BC0823B910509F44AC0833B91054E
:100CF00009F449C0843B910509F448C0853B91053E
:100D000009F447C0863B910509F446C0873B91052D
:100D100009F445C0883B910509F444C0893B91051D
:100D200009F443C08A3B910509F442C080E094E491
:100D3000089580E090E0089581E890E4089583E8C4
:100D400090E4089582EE94E4089589EE94E4089581
:100D50008AEE94E4089585EB94E4089586EB94E498
:100D6000089587EB94E408958CEC94E408958DEC59
:100D700094E4089583E895E408958AE895E4089555
:100D800082E995E4089584E995E4089581E296E482
:100D9000089583E296E4089584E296E4089585E256
:100DA00096E4089586E296E4089587E296E408952D
:100DB0008AE296E40895089524E5829FC0011124F3
:100DC000FC0126E0729FE00DF11D1124E60FF11DDC
:100DD000EE0FFF1FEF59FE4F859194910895880FF4
:100DE000991FFC01E553F040859194910895880F77
:100DF000991FFC01E55BFE4F85919491089524E5D0
:100E0000829FC0011124FC0146E0749FE00DF11D9A
:100E10001124E60FF11DEE0FFF1FEF59FE4F8591D4
:100E200094919C013A9521154FE1340708F425C1AE
:100E30003F512115304120F49F700E94F70608951C
:100E40009C0130532115304118F49927906C089576
:100E5000811520E5920769F40E94B1144FEF84E3F5
:100E60009CE0415080409040E1F700C000000C94AD
:100E7000681B813020E5920731F48091CC018160BC
:100E80008093CC0108959C0130552115304108F024
:100E90005CC0292F33272F70332721303105E9F427
:100EA000AC0164E0440F551F6A95E1F74427537085
:100EB000BC016370772702C0220F331F6A95E2F7E7
:100EC0003C68242B352B73E0880F991F7A95E1F746
:100ED00080769927822B932B08952230310529F4AF
:100EE000982F8827816F906A089523303105A1F4E7
:100EF000AC0133E0440F551F3A95E1F7407E57703F
:100F00008370992721E030E002C0220F331F8A95B9
:100F1000E2F7C9019C6816C02430310531F5AC01F7
:100F200023E0440F551F2A95E1F7407E57708370E8
:100F3000992721E030E002C0220F331F8A95E2F7A3
:100F4000C9019A68842B952B08959C01305721156F
:100F5000304118F49F70906208959C01305821151B
:100F6000304118F49F70906A0895803E9105E0F436
:100F7000803C910558F58133910509F46FC048F420
:100F80008932910509F463C08A32910509F46DC074
:100F900072C089339105E9F082389105D1F085332B
:100FA000910509F44DC067C0833E910581F138F485
:100FB000803E9105B9F0823E9105D9F05CC0863E35
:100FC000910561F1873E9105A1F155C00E94EF06A0
:100FD00008952091DE0120FD02C021FF4CC080EE6B
:100FE00090E049C08091DE0180FFF9CF89E390E075
:100FF00042C08091DE0182FF0EC08091DE0184FF3D
:1010000003C080E090E037C083EE90E034C0809170
:10101000DE0182FFF2CF82EE90E02DC08091DE01F2
:1010200083FF0BC08091DE0184FDEBCF87EE90E063
:1010300022C08091DE0183FFF5CF86EE90E01BC0D9
:101040008091DE0185FF07C089E290E014C08091A5
:10105000DE0185FFF9CF85E390E00DC08091DE01D0
:1010600086FF07C08AE290E006C08091DE0186FF1D
:10107000F9CF81E390E00E941B06089508958091C6
:1010800062010895CF93DF9300D01F92CDB7DEB7F2
:101090009C018091E401843019F593E099833B83AE
:1010A0002A839093E9008FEF9091E800815095FD9D
:1010B00006C095ED9A95F1F700008111F5CF80916A
:1010C000E80085FF0DC040E050E063E070E0CE0135
:1010D00001960E94AF0A8091E8008E778093E80025
:1010E0000F900F900F90DF91CF910895CF93DF93E2
:1010F00000D01F92CDB7DEB72091E401243021F556
:1011000022E029839B838A8383E08093E9008FEF29
:101110009091E800815095FD06C095ED9A95F1F704
:1011200000008111F5CF8091E80085FF0DC040E0FF
:1011300050E063E070E0CE0101960E94AF0A80911A
:10114000E8008E778093E8000F900F900F90DF916A
:10115000CF9108959C018091E4018430F9F482E0FC
:101160008093E9009FEF8091E800915085FD06C0D3
:1011700085ED8A95F1F700009111F5CF8091E80097
:1011800085FF0CC040E050E065E070E0C9010E94BE
:10119000AF0A8091E8008E778093E8000895CF939E
:1011A000DF93EC018091E401843009F046C0909116
:1011B0000C019923D9F090910D019923B9F08093F6
:1011C000E9008FEF9091E800815095FD06C095E110
:1011D0009A95F1F700008111F5CF8091E80085FF25
:1011E0002CC040E050E060E170E017C081E08093E7
:1011F000E9008FEF9091E800815095FD06C095EDD4
:101200009A95F1F700008111F5CF8091E80085FFF4
:1012100014C040E050E068E070E0CE010E94AF0AE8
:101220008091E8008E778093E80080E1FE01A2E5DE
:10123000B1E001900D928A95E1F7DF91CF91089589
:101240008091E301811109C00E94400C0E949D0C15
:101250008091E20084608093E20008951092E3019F
:10126000089508950C949E210E94FE1A0E94A421C4
:101270000E94480F0C943E0842E061EC81E00E941D
:10128000B90B42E061EC82E00E94B90B42E061ECF4
:1012900083E00E94B90B42E161EC84E00C94B90B4D
:1012A0008091E601833009F455C030F4813071F04B
:1012B000823009F48EC008958A3009F47AC08B30E8
:1012C00009F460C0893009F09CC020C08091E5011C
:1012D000813A09F096C08091E800877F8093E8000A
:1012E0008091E9019091EA01892B21F460E182E586
:1012F00091E003C060E080E090E070E00E94FA0AB4
:101300008091E8008B778093E80008958091E50153
:10131000813209F076C08091E9019091EA0100974D
:1013200019F0039709F06DC08091E800877F8093E2
:10133000E8008091E80082FD05C08091E401811100
:10134000F8CF5FC08091F100809362018091E80046
:101350008B7753C08091E501813A09F052C08091AA
:10136000E9019091EA01892B09F04BC08091E800D6
:10137000877F8093E8008091E80080FFFCCF809118
:101380000C0136C08091E5018132D9F58091E901E7
:101390009091EA01892BA9F58091E800877F8093DD
:1013A000E8000E94EE0B8091E70180930C010C9401
:1013B000B1148091E501813221F58091E800877FA9
:1013C0008093E8000E94EE0B8091E8018093630116
:1013D00008958091E501813AA1F48091E800877F2A
:1013E0008093E8008091E80080FFFCCF809163014A
:1013F0008093F1008091E8008E778093E8000C9450
:10140000EE0B089584B7877F84BF0FB6F894A89534
:1014100080916000886180936000109260000FBE30
:1014200090E080E80FB6F89480936100909361009B
:101430000FBE0E94970F0E94400C0E949D0C80914D
:10144000E20084608093E20078940E94280F0E945A
:10145000990F82E091E00E94430F0E948C218091BD
:10146000E401853069F40E94C01A8091E20188236A
:10147000B1F30E94EA1A882391F30E94990AEFCFF0
:101480000E949F0FECCF292F332723303105C9F05D
:1014900060F42130310581F02230310509F041C07E
:1014A0008DE690E02DED34E040C021323105E1F0D1
:1014B0002232310531F135C082E190E02AE435E095
:1014C00034C099278130910549F028F0029749F5F9
:1014D000E9EAF4E005C0E9EDF4E002C0E1ECF4E093
:1014E000849190E09F0121C06430D8F4E62FF0E0B1
:1014F000EE0FFF1FEE5DFE4F2081318189E090E00D
:1015000014C0643070F470E0FB01EE0FFF1FE65E64
:10151000FE4F20813181FB01EA5EFE4F808190E029
:1015200004C080E090E020E030E0FA0131832083C5
:10153000089580E189BD82E189BD09B400FEFDCF37
:101540008091D8008F7D8093D8008091E0008260E8
:101550008093E0008091E00081FDFCCF0895CF9260
:10156000DF92EF92FF920F931F93CF93DF93EC01E3
:101570008B016A010E940D0C811133C0C114D1048A
:1015800039F0F60180819181081B190BC80FD91F12
:10159000E12CF12C0115110519F18091E80085FD70
:1015A00016C08091E8008E778093E800C114D104C2
:1015B00049F0F60180819181E80EF91EF182E08206
:1015C00085E00FC00E940D0C882321F30AC0899189
:1015D0008093F10001501109FFEFEF1AFF0ADACFF3
:1015E00080E0DF91CF911F910F91FF90EF90DF90FE
:1015F000CF9008952091EB013091EC012617370729
:1016000048F06115710539F42091E8002E77209398
:10161000E80001C0B901FC0120E06115710579F114
:101620008091E4018823F1F18530F1F18091E800A7
:1016300083FD3CC08091E80082FD2EC08091E800CF
:1016400080FFEBCF2091F3008091F20090E0922B8D
:101650006115710551F08830910538F4219120937E
:10166000F100615071090196F3CF21E0089709F06C
:1016700020E08091E8008E778093E800CECF2111A2
:10168000CFCF0AC08091E401882361F0853061F0FA
:101690008091E80083FD0AC08091E80082FFF2CFCC
:1016A00080E0089582E0089583E0089581E0089540
:1016B0002091EB013091EC012617370748F06115B6
:1016C000710539F42091E8002E772093E80001C0DD
:1016D000B901FC0120E06115710591F18091E401EF
:1016E000882309F440C0853009F43FC08091E800A8
:1016F00083FD3DC08091E80082FD2FC08091E8000D
:1017000080FFE9CF2091F3008091F20090E0922BCE
:101710006115710559F08830910540F424912093AA
:10172000F1003196615071090196F2CF21E00897DE
:1017300009F020E08091E8008E778093E800CBCF1D
:101740002111CCCF0AC08091E401882361F085305B
:1017500061F08091E80083FD0AC08091E80082FF7B
:10176000F2CF80E0089582E0089583E0089581E05B
:101770000895982F973068F59093E900981739F0FD
:101780007091EC002091ED005091F00003C0242FE7
:10179000762F50E021FD02C09F5FECCF3091EB002F
:1017A0003E7F3093EB003091ED003D7F3093ED00B4
:1017B0003091EB0031603093EB007093EC0020939C
:1017C000ED005093F0002091EE0027FDE5CF80E082
:1017D00008958F708093E90081E008958091E5017C
:1017E00087FF11C08091E80082FD05C08091E4016F
:1017F0008111F8CF11C08091E8008B770BC08091E8
:10180000E401882349F08091E80080FFF8CF8091BF
:10181000E8008E778093E80008952091E4003091ED
:10182000E50095E64091EC00842F817040FF23C0D5
:101830008091E80080FD1DC08091E401882399F02B
:10184000853099F08091EB0085FD11C04091E40056
:101850005091E5002417350729F3915011F09A01B2
:10186000E1CF84E0089582E0089583E0089581E067
:10187000089580E008954091E80042FFDDCF08958B
:101880000E94AE0C0E94B60CE0EEF0E08081816018
:101890008083E8EDF0E080818F77808319BCA7ED2D
:1018A000B0E08C918E7F8C9380818F7E80831092AC
:1018B000E30108950F931F93CF93DF930E94AE0C23
:1018C0000E94B60CC8EDD0E088818F77888388812C
:1018D0008068888388818F7D888319BC1092E40199
:1018E0001092E0011092E2011092E10100EE10E08E
:1018F000F80180818B7F808388818160888342E0CA
:1019000060E080E00E94B90BE1EEF0E080818E7F24
:101910008083E2EEF0E08081816080838081886056
:101920008083F80180818E7F8083888180618883B5
:10193000DF91CF911F910F910895E8EDF0E0808144
:101940008F7E8083E7EDF0E080818160808384E09A
:1019500082BF81E08093E3010C945A0CE8EDF0E043
:1019600080818E7F80831092E20008951092DA00C9
:101970001092E10008951F920F920FB60F9211245A
:101980002F933F934F935F936F937F938F939F9387
:10199000AF93BF93EF93FF938091E10082FF0BC061
:1019A0008091E20082FF07C08091E1008B7F8093ED
:1019B000E1000E94270F8091DA0080FF1FC0809114
:1019C000D80080FF1BC08091DA008E7F8093DA0000
:1019D0008091D90080FF0DC080E189BD82E189BD81
:1019E00009B400FEFDCF81E08093E4010E9420094C
:1019F00005C019BC1092E4010E942E098091E100FB
:101A000080FF19C08091E20080FF15C08091E20044
:101A10008E7F8093E2008091E20080618093E200FB
:101A20008091D80080628093D80019BC85E08093B3
:101A3000E4010E9432098091E10084FF30C080916E
:101A4000E20084FF2CC080E189BD82E189BD09B438
:101A500000FEFDCF8091D8008F7D8093D8008091CB
:101A6000E1008F7E8093E1008091E2008F7E809381
:101A7000E2008091E20081608093E2008091E001C9
:101A8000882311F084E007C08091E30087FD02C045
:101A900081E001C083E08093E4010E9434098091D9
:101AA000E10083FF29C08091E20083FF25C080917F
:101AB000E100877F8093E10082E08093E40110924F
:101AC000E0018091E1008E7F8093E1008091E2004F
:101AD0008E7F8093E2008091E20080618093E2003B
:101AE00042E060E080E00E94B90B8091F0008860E5
:101AF0008093F0000E943109FF91EF91BF91AF9167
:101B00009F918F917F916F915F914F913F912F9115
:101B10000F900FBE0F901F9018951F920F920FB647
:101B20000F9211242F933F934F935F936F937F9363
:101B30008F939F93AF93BF93CF93DF93EF93FF93D5
:101B4000C091E900CF708091EC00D82FD17080FD5A
:101B5000D0E81092E9008091F000877F8093F00038
:101B600078940E94D10D1092E9008091F000886075
:101B70008093F000CD2BCF70C093E900FF91EF91DF
:101B8000DF91CF91BF91AF919F918F917F916F9195
:101B90005F914F913F912F910F900FBE0F901F902B
:101BA00018951F93CF93DF93CDB7DEB7AA970FB6E3
:101BB000F894DEBF0FBECDBFE5EEF1E08091F100FD
:101BC000819321E0ED3EF207C9F70E945009809110
:101BD000E80083FF24C18091E5019091E601492F3F
:101BE00050E04A30510508F01AC1FA01E15AFF4F9E
:101BF0000C943523803881F0823809F010C180912F
:101C0000E9018F708093E9008091EB0085FB8827C4
:101C100080F91092E90006C08091E1019091E20103
:101C2000911182609091E800977F9093E8008093F3
:101C3000F1001092F100C8C0282F2D7F09F0EFC0ED
:101C4000882319F0823061F0EAC08091E701813089
:101C500009F0E5C0933009F080E08093E2012BC0E9
:101C60008091E701811127C08091E9018F7009F40B
:101C7000D6C08093E9002091EB0020FF1CC0933078
:101C800021F48091EB00806214C09091EB00906190
:101C90009093EB0021E030E0A90102C0440F551FF2
:101CA0008A95E2F74093EA001092EA008091EB00F7
:101CB00088608093EB001092E9008091E800877FB4
:101CC00086C08111ACC01091E7011F778091E300BD
:101CD0008078812B8093E3008091E800877F809358
:101CE000E8000E94EE0B8091E80080FFFCCF80911D
:101CF000E30080688093E300111102C082E001C01C
:101D000083E08093E4018BC08058823008F087C064
:101D10008091E7019091E8018C3D53E0950779F5BA
:101D200083E08A838AE289834FB7F894DE011396B1
:101D300020E03EE051E2E32FF0E050935700E491C1
:101D400020FF03C0E295EF703F5FEF708E2F90E0B1
:101D5000EA3010F0C79601C0C0968D939D932F5F17
:101D6000243149F74FBF8091E800877F8093E800D6
:101D70006AE270E0CE0101960E94FA0A14C0AE0138
:101D80004F5F5F4F6091E9010E94430ABC01892BBC
:101D900009F445C09091E800977F9093E80089810D
:101DA0009A810E94580B8091E8008B778093E8001D
:101DB00036C08038A1F58091E800877F8093E800E5
:101DC0008091E0018093F1008091E8008E7780930C
:101DD000E8000E94EE0B23C0811121C08091E70131
:101DE0009091E80199270297D4F48091E800877FC9
:101DF0008093E8008091E7018093E0010E94EE0B60
:101E00008091E001811106C08091E30087FD02C04E
:101E100081E001C084E08093E4010E943C0980914C
:101E2000E80083FF0AC08091E800877F8093E80084
:101E30008091EB0080628093EB00AA960FB6F89435
:101E4000DEBF0FBECDBFDF91CF911F9108950895E2
:101E5000CF938091E4018823A1F0C091E900CF7075
:101E60009091EC00892F817090FD80E8C82B109232
:101E7000E9008091E80083FD0E94D10DCF70C093EE
:101E8000E900CF91089590936901809368010895C6
:101E9000E0916801F0916901309721F00190F081A3
:101EA000E02D099480E00895E0916801F0916901C6
:101EB000309721F00280F381E02D09940895E0919C
:101EC0006801F0916901309721F00480F581E02DDF
:101ED0000994089520916601309167012817390708
:101EE00071F09093670180936601E0916801F09131
:101EF0006901309721F00680F781E02D099408955B
:101F000020916401309165012817390771F0909391
:101F1000650180936401E0916801F0916901309757
:101F200021F00084F185E02D0994089508950C9422
:101F3000960F0E94041B0E9406050C94CA1BCF92A8
:101F4000DF92EF92FF920F931F93CF93DF93CDB762
:101F5000DEB72B970FB6F894DEBF0FBECDBF0E9441
:101F60001E058BE6C82E81E0D82E00E010E0E02EA2
:101F7000802F0E941406F60141916F01F82EF4267D
:101F8000B1F40F5F1F4F0E30110589F78FEF898372
:101F90008A831B820E940D1B8160782F9D838C8316
:101FA00049815A816B818D810E94421040C090917D
:101FB000CC0191FF04C08B870E941A068B8520E01C
:101FC00030E04F2D50E0922FBA01022E02C07595DD
:101FD00067950A94E2F760FF24C02E83EF8221E028
:101FE00030E0690102C0CC0CDD1C9A95E2F790E06C
:101FF0008C219D21892B09F420E028870E940D1B4C
:102000008160782F9A8789874E815F8168858A856C
:102010000E944210F801E559FE4F8081C826C08217
:1020200006C02F5F3F4F2630310569F6AACF0E94C8
:10203000B11E0E94480F90916A018917A1F00E9479
:10204000480F80936A012B960FB6F894DEBF0FBE3F
:10205000CDBFDF91CF911F910F91FF90EF90DF9057
:10206000CF900C943E082B960FB6F894DEBF0FBEAF
:10207000CDBFDF91CF911F910F91FF90EF90DF9037
:10208000CF900895CF93DF93CDB7DEB72B970FB6E0
:10209000F894DEBF0FBECDBF4F83588769877A871C
:1020A0008B87DE01119686E0FD0111928A95E9F792
:1020B00085E0FE01379601900D928A95E1F74981FE
:1020C0005A816B817C818D819E810E9445172B9660
:1020D0000FB6F894DEBF0FBECDBFDF91CF9108954C
:1020E000CF93C82F882309F4C1C0823859F40E94C5
:1020F000480F81FDBBC089E30E94E2190E949A1A31
:1021000089E30CC0833879F40E94480F80FDAEC08B
:1021100083E50E94E2190E949A1A83E50E94211A1F
:10212000CF910C949A1A843859F40E94480F82FD7A
:102130009DC087E40E94E2190E949A1A87E4EECFBC
:102140008CEF8C0F813A48F48C2F0E94F120811182
:102150008DC08C2F0E94E219E3CF80E28C0F883073
:1021600048F4C77081E001C0880FCA95EAF70E9461
:10217000631AD6CF8BE58C0F833078F4C53A29F0FB
:10218000C63A31F083E890E005C081E890E002C0F3
:1021900082E890E0CF910C946A0F88E58C0F833130
:1021A00008F064C0C83A39F1C93A41F1CA3A49F174
:1021B000CB3A51F1CC3A59F1CD3A61F1C03B69F1DA
:1021C000CE3A71F1CF3A79F1C13B81F1C23B89F14D
:1021D000C33B91F1C43B99F1C53BA1F1C63BA9F1C9
:1021E000C73BB1F1C83BB9F1C93BC1F1CA3BC9F129
:1021F00080E090E038C082EE90E035C089EE90E05B
:1022000032C08AEE90E02FC085EB90E02CC086EBC8
:1022100090E029C087EB90E026C08CEC90E023C0D2
:102220008DEC90E020C083E891E01DC08AE891E049
:102230001AC082E991E017C084E991E014C081E2FC
:1022400092E011C083E292E00EC084E292E00BC003
:1022500085E292E008C086E292E005C087E292E063
:1022600002C08AE292E0CF910C94800FCF91089542
:10227000882309F44BC0823859F40E94480F81FF2B
:1022800045C089E30E94E2190E949A1A89E30CC0B2
:10229000833871F40E94480F80FF38C083E50E94A4
:1022A000E2190E949A1A83E50E94211A0C949A1A44
:1022B000843859F40E94480F82FF28C087E40E94A6
:1022C000E2190E949A1A87E4EFCF9CEF980F913A97
:1022D00058F390E2980F983050F4877091E001C065
:1022E000990F8A95EAF7892F0E94691ADFCF9BE53B
:1022F000980F933020F480E090E00C946A0F885A95
:10230000833120F480E090E00C94800F08958823BE
:1023100021F00E94631A0C949A1A0895882321F0E0
:102320000E94691A0C949A1A0895BF92CF92DF9274
:10233000EF92FF920F931F93CF93DF9300D000D0C3
:1023400000D0CDB7DEB77C0185E0F701DE01119644
:1023500001900D928A95E1F7F70183819481892B91
:1023600009F4DDC2908181818F3F19F49F3F09F408
:10237000D6C2F7010281258122952F7099838A8325
:1023800089819A812E830E94A119182FB92E0E944B
:10239000A0190E946718EB2DE295EF704E2F50E0C8
:1023A000FA01E759FF4F2E810C9435238B2D807F46
:1023B0009B2D9F70F92E882319F0F29480EFF8225C
:1023C000002349F0FF2009F457C28F2D0E94731A91
:1023D0000E949A1A51C2812F0E943811FF2009F4DD
:1023E0009EC28F2D0E94791A26960FB6F894DEBFF2
:1023F0000FBECDBFDF91CF911F910F91FF90EF9056
:10240000DF90CF90BF900C949A1A3B2D307F8B2D8C
:102410008F70303211F08295807F112319F01130C6
:1024200021F12CC00023B9F0222309F490C12130FE
:1024300009F08DC126960FB6F894DEBF0FBECDBF52
:10244000DF91CF911F910F91FF90EF90DF90CF9090
:10245000BF900C94831A222319F0213009F45FC233
:102460008E830E94861A8E8186C1002321F022303D
:1024700008F055C26CC1211152C27DC1002321F068
:10248000222309F464C1F8C1222309F474C109C2EA
:102490008B2D86958695837019F08130D1F03FC2DF
:1024A000002321F0812F9B2D937002C080E090E0EB
:1024B00026960FB6F894DEBF0FBECDBFDF91CF9149
:1024C0001F910F91FF90EF90DF90CF90BF900C94F1
:1024D0006A0F002321F0812F9B2D937002C080E0B2
:1024E00090E026960FB6F894DEBF0FBECDBFDF9109
:1024F000CF911F910F91FF90EF90DF90CF90BF9001
:102500000C94800F812F002319F00E94B91D02C086
:102510000E94211E26960FB6F894DEBF0FBECDBFD7
:10252000DF91CF911F910F91FF90EF90DF90CF90AF
:10253000BF900C94A61E8B2D837009F075C00111FD
:10254000EEC1812F829586958770880F880F912F15
:102550009F70C92ED12CE12CF12C082E04C0CC0C7C
:10256000DD1CEE1CFF1C0A94D2F714FF12C00FE012
:1025700010E020E030E004C0000F111F221F331FC5
:102580008A95D2F7C901B8016095709580959095AC
:1025900003C060E070E0CB014B2D4695469543703B
:1025A0004230C1F060F56C297D298E299F29413088
:1025B00051F126960FB6F894DEBF0FBECDBFDF9166
:1025C000CF911F910F91FF90EF90DF90CF90BF9030
:1025D0000C948E186C297D298E299F2926960FB67A
:1025E000F894DEBF0FBECDBFDF91CF911F910F9149
:1025F000FF90EF90DF90CF90BF900C94AA180E94AC
:102600008E18C701B60126960FB6F894DEBF0FBE2E
:10261000CDBFDF91CF911F910F91FF90EF90DF9091
:10262000CF90BF900C947218002319F08B2D8170FD
:1026300001C08695882309F472C1812F8295869501
:102640008770880F880F912F9F70C92ED12CE12C95
:10265000F12C082E04C0CC0CDD1CEE1CFF1C0A94CF
:10266000D2F714FF12C00FE010E020E030E004C009
:10267000000F111F221F331F8A95D2F7C901B8011D
:10268000609570958095909503C060E070E0CB01F7
:102690004B2D4695469543704230C1F060F56C294C
:1026A0007D298E299F29413051F126960FB6F89445
:1026B000DEBF0FBECDBFDF91CF911F910F91FF9075
:1026C000EF90DF90CF90BF900C9468196C297D2912
:1026D0008E299F2926960FB6F894DEBF0FBECDBF78
:1026E000DF91CF911F910F91FF90EF90DF90CF90EE
:1026F000BF900C9484190E946819C701B6012696F0
:102700000FB6F894DEBF0FBECDBFDF91CF911F9102
:102710000F91FF90EF90DF90CF90BF900C944C19E9
:10272000103FD1F118F4103E50F4A1C0123F09F44B
:1027300063C008F44CC0133F09F473C098C01F7005
:102740008B2D8F710023A1F00E94E518812F269612
:102750000FB6F894DEBF0FBECDBFDF91CF911F91B2
:102760000F91FF90EF90DF90CF90BF900C94871166
:102770000E940619812F26960FB6F894DEBF0FBE71
:10278000CDBFDF91CF911F910F91FF90EF90DF9020
:10279000CF90BF900C948E110023A9F02111BFC0DF
:1027A0008B2D8F7126960FB6F894DEBF0FBECDBF6E
:1027B000DF91CF911F910F91FF90EF90DF90CF901D
:1027C000BF900C942B19223008F0A9C0E9CF002348
:1027D000A9F08B2D8F7126960FB6F894DEBF0FBE31
:1027E000CDBFDF91CF911F910F91FF90EF90DF90C0
:1027F000CF90BF900C94E518002359F38B2D8F7167
:1028000026960FB6F894DEBF0FBECDBFDF91CF91F5
:102810001F910F91FF90EF90DF90CF90BF900C949D
:102820000619002399F08B2D8F7126960FB6F89418
:10283000DEBF0FBECDBFDF91CF911F910F91FF90F3
:10284000EF90DF90CF90BF900C94D01826960FB6E3
:10285000F894DEBF0FBECDBFDF91CF911F910F91D6
:10286000FF90EF90DF90CF90BF900C94C61800239C
:10287000A9F0222309F4ADCF812F26960FB6F89444
:10288000DEBF0FBECDBFDF91CF911F910F91FF90A3
:10289000EF90DF90CF90BF900C947010222309F43A
:1028A000ADCF812F26960FB6F894DEBF0FBECDBFF9
:1028B000DF91CF911F910F91FF90EF90DF90CF901C
:1028C000BF900C9438114B2D4F70612FC7010E949F
:1028D000950326960FB6F894DEBF0FBECDBFDF91ED
:1028E000CF911F910F91FF90EF90DF90CF90BF900D
:1028F0000C94EA174B2D4F70612FC70126960FB627
:10290000F894DEBF0FBECDBFDF91CF911F910F9125
:10291000FF90EF90DF90CF90BF900C94DB0626964F
:102920000FB6F894DEBF0FBECDBFDF91CF911F91E0
:102930000F91FF90EF90DF90CF90BF9008950E948D
:10294000801A0E94551A0E949A1A0E94561F0E94CD
:10295000A61E80E090E00E946A0F80E090E00C9458
:10296000800F0E94701A0C949F140E94A119292FA5
:1029700022952F702C3030F42A3048F42250223027
:1029800078F405C02C3041F02F3031F009C0803E82
:1029900048F0803F29F406C093FB882780F908950A
:1029A00080E0089581E00895CF93DF9300D000D0B8
:1029B0001F92CDB7DEB70F900F900F900F900F9032
:1029C000DF91CF910895CF93DF9300D000D000D056
:1029D000CDB7DEB726960FB6F894DEBF0FBECDBFDB
:1029E000DF91CF9108951F93CF93DF93C091790129
:1029F00016E080917A01C81799F0D0E01C9FF00191
:102A00001D9FF00D1124E558FE4F408151816281D8
:102A10007381848195810E94E3142196C770E9CF68
:102A2000DF91CF911F9108954091AB015091AC017E
:102A30006091AD017091AE018091AF019091B001B4
:102A40000C94E3148091B00182958F7009F054C00A
:102A50008091AD01882309F44FC080917901A09144
:102A60007A014091AE015091AF016091AB0170913C
:102A7000AC01B6E08A1709F43FC090E0411551055A
:102A8000C1F17F3F11F46F3FA1F1B89FF001B99FF1
:102A9000F00D1124E558FE4F218127132AC0208113
:102AA000261327C02281211124C0238134812417B9
:102AB000350710F421503109241B350B283C310512
:102AC000C0F42091B0012F7020612093B00126E066
:102AD000289FF001299FF00D1124E058FE4F8081BE
:102AE0008F70806180838BEA91E00E9495110C9435
:102AF000F31401968770BECF0895CF92DF92EF92C4
:102B0000FF920F931F93CF93DF93CDB7DEB76297FA
:102B10000FB6F894DEBF0FBECDBF8C0185E0F80183
:102B2000DE011D9601900D928A95E1F7D8014C9136
:102B300011965C91119712966C918091AE019091D3
:102B4000AF01009709F475C13091AB017091AC01F0
:102B50007F3F19F43F3F09F46CC1F801C380D48072
:102B6000E090AD01EE2009F4BEC02091B001C8167E
:102B7000D90628F0D601A81BB90BCD0104C0809559
:102B800090958C0D9D1DFF24F394883C910578F061
:102B9000F12C207F09F0C4C07C2DD98AC88A89898C
:102BA0000E94D4148BEA91E00E949511AFC0822F4D
:102BB000807F09F045C0571313C0431311C0611142
:102BC0000FC02F7020612093B0010E9414158BEA72
:102BD00091E00E9495118091B001F80185832EC08B
:102BE000CD2819F15F3F11F44F3FF9F0F62E611136
:102BF0001CC08091790120917A0136E0821709F496
:102C00005BC090E0389FF001399FF00D1124E5582A
:102C1000FE4F7181571306C07081471303C0728144
:102C2000711103C001968770E9CFF62E662309F46F
:102C30001CC18091B00181608093B001F12C15C15D
:102C4000571309C0431307C0611105C08091B0013B
:102C5000F8018583C8C04D875E878D859E856A8B08
:102C60000E94B5146A898823D1F16623C1F12091AD
:102C7000B001822F82958F7090E0029774F080915E
:102C8000AB019091AC0198878F831986DB86CA8649
:102C90002C87CE0107960E94951186E0F801ABEAD9
:102CA000B1E001900D928A95E1F70E9422150E94F1
:102CB0001415FF24F394D9C04D875E878D859E85BA
:102CC0000E94A119292F22952F70223008F0C1C02F
:102CD0009F7009F0BBC0805E883008F4C6C0C80190
:102CE0000E949511E6CFC816D90608F453C0F60124
:102CF000E81BF90BCF01883C910508F450C0F12C7A
:102D00007C2DD98AC88A89890E94D414EBEAF1E023
:102D100086E0DF011D928A95E9F70E941415A5C08F
:102D2000571314C0431312C0611110C08091B00139
:102D3000F8018583C8010E94951186E0EBEAF1E075
:102D4000DF011D928A95E9F7FE2C8FC04D875E87C3
:102D50008D859E856A8B0E94B5146A89882309F443
:102D6000BECF662309F4BBCF2091B001822F82959C
:102D70008F7090E002970CF490CF8091AB0190910E
:102D8000AC019A8389831B82DD82CC822E83CE01A3
:102D9000019681CF809590958C0D9D1DACCFF62E20
:102DA000662309F49CCF571333C0431331C02091DD
:102DB000B00120FD24C0822F82958F70482F50E0F3
:102DC00041155105E1F0D80115962C9315974F3018
:102DD000510549F08F5F982F9295907F822F8F70C9
:102DE000892B15968C93C8010E94951186E0F801F5
:102DF000ABEAB1E001900D928A95E1F78ECF86E0C3
:102E0000F801ABEAB1E001900D928A95E1F72DC08F
:102E10004D875E878D859E850E94B51481113DCFBB
:102E20008091B00181608093B001C8010E9495112A
:102E30001CC0662309F453CF4D875E878D859E8520
:102E40000E94B514882309F44ACF27CF811143CFBC
:102E50000CC0243008F043CF9F7009F43CCFD80158
:102E600015969C91907F09F036CF8F2D62960FB604
:102E7000F894DEBF0FBECDBFDF91CF911F910F91B0
:102E8000FF90EF90DF90CF9008951F93CF93DF9343
:102E9000CDB7DEB72C970FB6F894DEBF0FBECDBF0F
:102EA0004F83588769877A878B879C87CE010796DF
:102EB0000E947D15882371F08A859B85892B09F4F2
:102EC00041C088858F3F09F065C08F818F3F09F031
:102ED00061C038C086E0FE013796DE011196019090
:102EE0000D928A95E1F76A857B856115710551F12F
:102EF000FF81E885EF3F11F4FF3F21F120917A0136
:102F000030E0C9010196877099274091790150E01E
:102F10008417950709F447C0F983EA837D836C839E
:102F200096E0929FD001939FB00D1124A558BE4FFB
:102F3000FE01319601900D929A95E1F780937A0106
:102F40000E94F31416E08091790190917A0189171B
:102F5000B9F1189FC001112485589E4F0E947D151C
:102F6000882371F1E09179011E9FF0011124E55849
:102F7000FE4F4081518162817381848195810E94DD
:102F8000E3148091790190E00196877099278093EE
:102F90007901D9CF4F81588569857A858B859C8544
:102FA0000E94E314CFCF0E94B11410927A011092C4
:102FB0007901EBEAF1E086E0DF011D928A95E9F7FD
:102FC0002C960FB6F894DEBF0FBECDBFDF91CF9128
:102FD0001F910895EF92FF920F931F93CF93DF936A
:102FE0008C01892B09F46CC0F12CEE24E394E801E8
:102FF0002196F8018491843740F4843008F051C060
:10300000813081F0823019F15BC0853709F444C00A
:10301000A8F19CE7980F903708F052C08F770E9474
:10302000381141C00E5F1F4FFE01849190E2980F4E
:10303000983050F48770FE2D01C0FF0F8A95EAF793
:103040008F2F0E94731A14C00E9470102DC00E5F43
:103050001F4FFE01849190E2980F983060F48770C2
:10306000FE2D01C0FF0F8A95EAF78F2F0E94791A73
:103070000E949A1A19C00E94381116C00E5F1F4F85
:10308000FE01C491CC2381F08FE99FE00197F1F715
:1030900000C00000C150F6CF0E5F1F4FFE01F4903C
:1030A00003C00E9470108E018F2D882309F49FCFDA
:1030B000EFE9FFE03197F1F700C000008150F5CF54
:1030C000DF91CF911F910F91FF90EF900895089598
:1030D0006093B5017093B6018093B7019093B801E6
:1030E0000C949F140F931F930091B5011091B6019A
:1030F0002091B7013091B801DC01CB01802B912BDD
:10310000A22BB32B8093B5019093B601A093B70186
:10311000B093B8011F910F910C949F140F931F93BC
:103120000091B5011091B6012091B7013091B8011D
:10313000DC01CB0180239123A223B3238093B5012B
:103140009093B601A093B701B093B8011F910F916E
:103150000C949F140F931F930091B5011091B60129
:103160002091B7013091B801DC01CB018027912774
:10317000A227B3278093B5019093B601A093B7011E
:10318000B093B8011F910F910C949F141092B1014C
:103190001092B2011092B3011092B4010C949F14DA
:1031A00041E050E060E070E004C0440F551F661F2E
:1031B000771F8A95D2F74093B1015093B201609383
:1031C000B3017093B4010C949F1441E050E060E0AF
:1031D00070E004C0440F551F661F771F8A95D2F711
:1031E0008091B1019091B201A091B301B091B4016D
:1031F000482B592B6A2B7B2B4093B1015093B20182
:103200006093B3017093B4010C949F1441E050E0BB
:1032100060E070E004C0440F551F661F771F8A9559
:10322000D2F740955095609570958091B10190913D
:10323000B201A091B301B091B401482359236A238C
:103240007B234093B1015093B2016093B30170931B
:10325000B4010C949F1441E050E060E070E004C0C1
:10326000440F551F661F771F8A95D2F78091B101D1
:103270009091B201A091B301B091B40148275927B0
:103280006A277B274093B1015093B2016093B30149
:103290007093B4010C949F140F931F930091B1018C
:1032A0001091B2012091B3013091B401DC01CB0146
:1032B000802B912BA22BB32B8093B1019093B20161
:1032C000A093B301B093B4011F910F910C949F147C
:1032D0000F931F930091B1011091B2012091B3019E
:1032E0003091B401DC01CB0180239123A223B323CD
:1032F0008093B1019093B201A093B301B093B40154
:103300001F910F910C949F140F931F930091B10183
:103310001091B2012091B3013091B401DC01CB01D5
:1033200080279127A227B3278093B1019093B20100
:10333000A093B301B093B4011F910F910C949F140B
:103340000895CF92DF92EF92FF920F931F93CF9346
:10335000DF938C01C090B101D090B201E090B30135
:10336000F090B4018091B5019091B601A091B701A0
:10337000B091B801C82AD92AEA2AFB2ACFE1D0E0C5
:10338000D701C6010C2E04C0B695A79597958795D1
:103390000A94D2F780FF07C0B8018C2F0E94FF0665
:1033A0008130910531F4219758F7B80180E00E94EF
:1033B000FF06DF91CF911F910F91FF90EF90DF906B
:1033C000CF90089590910C019923F1F090910D0107
:1033D0009923D1F0982F9695969596959F3080F5E4
:1033E000E0910E01F0910F01E90FF11D877021E0CE
:1033F00030E0A90102C0440F551F8A95E2F7CA01C7
:103400009181892B8183089520910E0130910F01C4
:10341000F90132969FEF40E05191851789F09F3F67
:1034200019F4511101C0942F4F5F4E30A9F79F3FFF
:1034300039F0F901E90FF11D97FDFA95828308959E
:10344000089590910C019923F9F090910D01992321
:10345000D9F0982F9695969596959F3028F5E091FE
:103460000E01F0910F01E90FF11D877021E030E0AE
:10347000A90102C0440F551F8A95E2F7CA01809541
:10348000918189238183089520910E0130910F014C
:10349000F9013296205F3F4F9081891301C010825D
:1034A0003196E217F307C1F7089581E090E0E091CB
:1034B0000E01F0910F01E80FF91F10820196803183
:1034C0009105A9F708959091CB01892B8093CB01A9
:1034D000089580959091CB0189238093CB01089525
:1034E0001092CB0108959091CA01892B8093CA0153
:1034F000089580959091CA0189238093CA01089507
:103500001092CA0108958093B90108951092B901EB
:10351000089580910E0190910F01FC0131969C015C
:10352000205F3F4F80E0919191118F5FE217F30789
:10353000D1F70895E0910E01F0910F018091CB0138
:103540008083E0910E01F0910F0190818091CA017A
:10355000892B80838091B901882361F0E0910E016D
:10356000F0910F019081892B80830E94891A81112B
:103570001092B90180910E0190910F010C94540F9B
:103580008091E401843011F120E488E190E00FB6ED
:10359000F894A895809360000FBE2093600083B7D5
:1035A000817F846083BF83B7816083BF789488956F
:1035B00083B78E7F83BF0FB6F894A8958091600083
:1035C000886180936000109260000FBE0895089596
:1035D0000C94E71ACF930E94E81A0E941E050E94DD
:1035E000E71AC0E08C2F0E941406811104C0CF5F3F
:1035F000CE30C1F701C081E0CF9108950E94B1148F
:103600000E94480F0C943E0882E084BD93E095BD73
:103610009AEF97BD80936E0008952FB7F89480912C
:10362000CD019091CE01A091CF01B091D0012FBFDB
:103630000895CF92DF92EF92FF920F931F932FB7CF
:10364000F8944091CD015091CE016091CF017091DD
:10365000D0012FBF6A017B01EE24FF248C0120E002
:1036600030E0C016D106E206F30610F441505109CD
:103670009A01281B390BC9011F910F91FF90EF9000
:10368000DF90CF9008951F920F920FB60F921124E2
:103690008F939F93AF93BF938091CD019091CE0173
:1036A000A091CF01B091D0010196A11DB11D8093D1
:1036B000CD019093CE01A093CF01B093D001BF91E3
:1036C000AF919F918F910F900FBE0F901F90189503
:1036D0000E94400CF8942FEF87EA91E62150804039
:1036E0009040E1F700C0000087E090EBDC018093A0
:1036F000ED019093EE01A093EF01B093F0019CE0F7
:1037000088E10FB6F894A895809360000FBE90935F
:103710006000FFCFEF92FF920F931F93CF93DF9341
:10372000D82FC0E08C2F0E94140600E010E0E82E95
:10373000F12CC701002E02C0959587950A94E2F7F7
:1037400080FD06C00F5F1F4F0630110591F709C0BD
:10375000602F7C2F80E00E94DC068D13F3CF81E088
:1037600004C0CF5FCE30F1F680E0DF91CF911F91A2
:103770000F91FF90EF900895CF93C82F8CE20E9495
:103780008A1B882321F08C2FCF910C948A1B80E018
:10379000CF910895CF930E94111D811102C00E9404
:1037A000F71CC5E6C15049F00E941E058FE39CE955
:1037B0000197F1F700C00000F5CF89E20E94BC1B21
:1037C000811113C18AE20E94BC1B81110E94F71C67
:1037D00085E00E94BC1B81110E94681B0E941C1D79
:1037E0008093CC0187E00E94BC1B8823A9F18BE168
:1037F0000E94BC1B882351F08091CC0181FB2227C1
:1038000020F991E0922790FB81F90EC08EE00E9492
:10381000BC1B882361F08091CC0182FB222720F918
:1038200091E0922790FB82F98093CC0115C080E152
:103830000E94BC1B9091CC01882341F093FB22276E
:1038400020F981E0822780FB93F904C0892F8095BD
:1038500080FB90F99093CC018091CC010E94201DB7
:103860000E942E1D8093DE0180EE0E94BC1B8823E7
:1038700041F08091DE01982F909590FB80F9809324
:10388000DE0189E30E94BC1B882359F08091DE0190
:1038900081FB222720F991E0922790FB81F9809308
:1038A000DE0182EE0E94BC1B882359F08091DE016C
:1038B00082FB222720F991E0922790FB82F98093E6
:1038C000DE0186EE0E94BC1B882359F08091DE0148
:1038D00083FB222720F991E0922790FB83F98093C4
:1038E000DE0183EE0E94BC1B882359F08091DE012B
:1038F00084FB222720F991E0922790FB84F98093A2
:10390000DE0185E30E94BC1B882359F08091DE0113
:1039100085FB222720F991E0922790FB85F980937F
:10392000DE0181E30E94BC1B882359F08091DE01F7
:1039300086FB222720F991E0922790FB86F980935D
:10394000DE0181E10E94BC1B882359F08091DE01D9
:1039500087FB222720F991E0922790FB87F980933B
:10396000DE018091DE010E94321D8091DE0187FB25
:10397000882780F980930D0187E20E94BC1BC82F25
:103980008EE10E94BC1B8111C2608FE10E94BC1BB2
:103990008111C46080E20E94BC1B8111C86081E279
:1039A0000E94BC1B8111C06182E20E94BC1B81117C
:1039B000C06283E20E94BC1B8111C06484E20E9449
:1039C000BC1B882311F0C06802C0CC2329F08C2FC7
:1039D0000E94291D6C2F03C00E94251D682F70E0D6
:1039E00080E090E0CF910C946818CF9108956DEE2F
:1039F0007EEF80E090E00E946B2360E082E090E048
:103A00000E945D2360E083E090E00E945D2360E01F
:103A100084E090E00E945D2360E085E090E00C94FB
:103A20005D2380E090E00E94572321E08D3E9E4F71
:103A300009F020E0822F089582E090E00C944F235B
:103A4000682F82E090E00C945D2383E090E00C947A
:103A50004F23682F83E090E00C945D2384E090E096
:103A60000C944F23682F84E090E00C945D238091A8
:103A7000D30180FF0BC06091130185E0689FB00106
:103A8000112475956795759567952BC081FF09C0C1
:103A90006091130185E0689FB001112475956795C9
:103AA00020C082FF07C06091130185E0689FB001CC
:103AB000112417C09091D4019923D1F06091120183
:103AC000961788F72091130185E0289F9001112413
:103AD000929FA001939F500D112470E0CA010E9493
:103AE00021236038710540F46115710519F406C091
:103AF00065E070E0862F08958FE7089581E00895CE
:103B00008091D30180FF08C06091110170E075952C
:103B100067957595679521C081FF06C06091110179
:103B200070E07595679519C082FF04C0609111011E
:103B300070E010C09091D401992399F06091100128
:103B40009617A0F780911101899FC001112470E0A0
:103B50000E9421236038710540F46115710519F444
:103B600006C061E070E0862F08958FE7089581E038
:103B70000895803F21F40E94371D819504C0813F44
:103B800029F40E94371D8093D7010895823F21F4C4
:103B90000E94371D819504C0833F29F40E94371D80
:103BA0008093D6010895893F19F40E94801D05C0B5
:103BB0008A3F31F40E94801D81958093D801089539
:103BC0008B3F21F40E94801D819504C08C3F29F415
:103BD0000E94801D8093D9010895843F21F4809133
:103BE000D501816017C0853F21F48091D5018260A5
:103BF00011C0863F21F48091D50184600BC0873FBE
:103C000021F48091D501886005C0883F31F480910E
:103C1000D50180618093D50108958D3F21F4809175
:103C2000D30181600BC08E3F21F48091D30182606B
:103C300005C08F3F29F48091D30184608093D30124
:103C40000895803F39F48091D70187FF6CC01092AE
:103C5000D70169C0813F29F48091D7011816BCF3C0
:103C600062C09091D601823F29F497FF5CC0109208
:103C7000D60159C0833F19F41916CCF354C0893FBB
:103C800041F48091D80118160CF04DC01092D80163
:103C90004AC08A3F29F48091D80187FF44C0F6CFFB
:103CA0008B3F39F48091D90187FF3DC01092D90133
:103CB0003AC08C3F29F48091D9011816BCF333C067
:103CC000843F21F48091D5018E7F17C0853F21F478
:103CD0008091D5018D7F11C0863F21F48091D5015F
:103CE0008B7F0BC0873F21F48091D501877F05C072
:103CF000883F31F48091D5018F7E8093D50113C028
:103D00008D3F21F48091D3018E7F0BC08E3F21F433
:103D10008091D3018D7F05C08F3F29F48091D3011D
:103D20008B7F8093D3018091D60181110EC0809149
:103D3000D70181110AC08091D801811106C08091FC
:103D4000D901811102C01092D401089585ED91E04E
:103D50000E945F0F0E940D1B9093D2018093D101AE
:103D600008951F93CF93DF938091D1019091D20159
:103D70000E94191BAC019091D401992321F020914C
:103D8000140130E006C0209115018AE0289F9001BF
:103D900011244217530708F485C08091D601C091C1
:103DA000D701D091D8011091D901811107C0C1115B
:103DB00075C0D11173C0111171C074C09F3F19F04B
:103DC0009F5F9093D401181624F40E94371D8093AE
:103DD000D6018091D60187FF05C00E94371D8195CD
:103DE0008093D6011C1624F40E94371D8093D701BE
:103DF0008091D70187FF05C00E94371D8195809370
:103E0000D7016091D601662331F1C091D701CC234F
:103E100011F1062E000C770B880B990B0E942822BB
:103E200023E333E343E35FE30E948C220E94F0210B
:103E30006093D6016C2FCC0F770B880B990B0E94E7
:103E4000282223E333E343E35FE30E948C220E94B2
:103E5000F0216093D7011D1624F40E94801D8093E9
:103E6000D8018091D80187FF05C00E94801D8195EF
:103E70008093D801111624F40E94801D8093D901EB
:103E80008091D90187FF05C00E94801D8195809394
:103E9000D901DF91CF911F910C94A61E9F3F09F08D
:103EA0008FCFA0CFDF91CF911F910895E5EDF1E085
:103EB00085E0DF011D928A95E9F71092D4011092F6
:103EC000D3010895833081F128F4813059F0823094
:103ED000D1F00895853009F449C0B8F1863009F46D
:103EE00056C0089580911501262F30E0280F311D0E
:103EF0002F3F310524F4680F6093150108958FEF6B
:103F000080931501089580911401262F30E0280F29
:103F1000311D2F3F310524F4680F6093140108957B
:103F20008FEF80931401089580911301262F30E0C4
:103F3000280F311D2F3F310524F4680F60931301C2
:103F400008958FEF80931301089580911201262F19
:103F500030E0280F311D2F3F310524F4680F6093A6
:103F6000120108958FEF809312010895809111013D
:103F7000262F30E0280F311D2F3F310524F4680F24
:103F80006093110108958FEF80931101089580913E
:103F90001001262F30E0280F311D2F3F310524F46A
:103FA000680F6093100108958FEF809310010895BA
:103FB000833011F128F4813049F0823091F0089576
:103FC000853081F120F18630C1F10895809115018D
:103FD000681720F4861B809315010895109215012F
:103FE000089580911401681720F4861B80931401B2
:103FF000089510921401089580911301681720F418
:10400000861B8093130108951092130108958091E7
:104010001201681720F4861B8093120108951092F4
:104020001201089580911101681720F4861B809376
:1040300011010895109211010895809110016817DF
:1040400020F4861B809310010895109210010895AA
:104050000F931F938D3109F46BC008F03FC08E3071
:1040600009F47DC0C0F4873009F46EC068F486306E
:1040700009F0AFC08091CC01817F8E7F8093CC010D
:1040800081E08093DB01A6C0883009F458C08B30F2
:1040900009F49BC09EC0863109F497C078F4803142
:1040A00009F470C0813109F094C00E94B11490915C
:1040B0000D0181E0892780930D0187C0893109F4C2
:1040C00084C08B3109F085C08091CC0181FB22270F
:1040D00020F991E0922790FB81F94AC0853309F4D9
:1040E0005BC048F4873209F457C008F45AC08932DB
:1040F00009F452C06EC0833438F48A3308F067C0C4
:10410000883309F462C065C0833409F445C088343B
:1041100009F05FC00E94B1140FEF13ED20E30150CE
:1041200010402040E1F700C000000E94681B4DC015
:104130000E94AA210E94480F0E943E0846C00E9489
:104140001C1D0E942E1D41C09091CC01892F8170B1
:1041500090FF12C0917F9E7F9093CC013BC08091D5
:10416000CC0182FB222720F991E0922790FB82F973
:104170008093CC01992349F18091CC018160809397
:10418000CC0123C08091CC0183FB222720F991E050
:10419000922790FB83F9ECCF61E070E080E090E043
:1041A00010C08D5141E050E060E070E08A019B0159
:1041B00004C0000F111F221F331F8A95D2F7C901B7
:1041C000B8010E9468180E94B11481E003C08953AD
:1041D000E9CF80E01F910F91089580E008950C943D
:1041E000ED20CF93C82F8091DB01813079F018F05A
:1041F0008230E9F187C0E0910E01F0910F018081DA
:10420000813169F0823209F07FC009C0E0910E016E
:10421000F0910F018081813111F0823261F48C2F95
:104220000E94EF20811104C08C2F0E9428201DC005
:1042300081E090E01AC08C2F0E94ED20811114C003
:10424000C43179F048F4CB3079F0C03109F060C066
:1042500082E08093DB0108C0C93219F0C83321F035
:1042600057C01092DB0154C081E0817053C0C93245
:1042700089F118F5C43171F1A8F4C73009F046C0CE
:104280008AE08093150194E19093140193E0909358
:1042900013018093120188E08093110188E28093DA
:1042A000100134C0CE51C63088F5EC2FF0E0E65D49
:1042B000FE4F80818093DA0129C0CE34E9F020F4EA
:1042C000CB3421F56AE013C0C13579F0C235F1F481
:1042D00061E00DC08091DA01882319F01092DA01B3
:1042E00015C081E08093DB0115C061E006C08091BC
:1042F000DA010E94621F0AC06AE08091DA010E941E
:10430000D81F04C01092DB0180E004C081E002C02D
:1043100080E0ABCFCF910895E1E8F0E08081886044
:1043200080838081816080838FB7F89493E090933D
:10433000890090ED909388008FBF0895EFE6F0E03C
:104340008081826080830895EFE6F0E080818D7F38
:1043500080830895EFE6F0E0908182E089278083F2
:1043600008951F920F920FB60F9211242F933F932F
:104370004F935F936F937F938F939F93AF93BF936D
:10438000EF93FF938091DC019091DD010196909372
:10439000DD018093DC01811103C082E00E943E08B0
:1043A000E091DD01E695E695F0E0E95AF94FE491F8
:1043B0008091DC018E1303C080E00E943E08FF91D3
:1043C000EF91BF91AF919F918F917F916F915F918D
:1043D0004F913F912F910F900FBE0F901F90189506
:1043E0000E94F7216894B1110C94862208950E94CE
:1043F0006B2288F09F5798F0B92F9927B751B0F0EA
:10440000E1F0660F771F881F991F1AF0BA95C9F758
:1044100014C0B13091F00E948522B1E008950C944F
:104420008522672F782F8827B85F39F0B93FCCF302
:10443000869577956795B395D9F73EF490958095D5
:10444000709561957F4F8F4F9F4F0895E89409C0F5
:1044500097FB3EF490958095709561957F4F8F4FB7
:104460009F4F9923A9F0F92F96E9BB279395F695CD
:10447000879577956795B795F111F8CFFAF4BB0F4B
:1044800011F460FF1BC06F5F7F4F8F4F9F4F16C0AF
:10449000882311F096E911C0772321F09EE8872F39
:1044A000762F05C0662371F096E8862F70E060E0F5
:1044B0002AF09A95660F771F881FDAF7880F96956E
:1044C000879597F9089557FD9058440F551F59F057
:1044D0005F3F71F04795880F97FB991F61F09F3FF1
:1044E00079F087950895121613061406551FF2CF1A
:1044F0004695F1DF08C0161617061806991FF1CF6A
:1045000086957105610508940895E894BB27662790
:104510007727CB0197F908950E949F220C941023CE
:104520000E94022338F00E94092320F0952311F005
:104530000C94F9220C94FF2211240C9486220E94E0
:10454000632270F3959FC1F3950F50E0551F629F52
:10455000F001729FBB27F00DB11D639FAA27F00DDC
:10456000B11DAA1F649F6627B00DA11D661F829F03
:104570002227B00DA11D621F739FB00DA11D621FE8
:10458000839FA00D611D221F749F3327A00D611D05
:10459000231F849F600D211D822F762F6A2F1124E7
:1045A0009F5750409AF0F1F088234AF0EE0FFF1F1A
:1045B000BB1F661F771F881F91505040A9F79E3F71
:1045C000510580F00C94F9220C9486225F3FE4F3AD
:1045D000983ED4F3869577956795B795F795E795C7
:1045E0009F5FC1F7FE2B880F911D9695879597F9D0
:1045F000089597F99F6780E870E060E008959FEF65
:1046000080EC089500240A94161617061806090669
:10461000089500240A941216130614060506089538
:10462000092E0394000C11F4882352F0BB0F40F4C0
:10463000BF2B11F460FF04C06F5F7F4F8F4F9F4F00
:10464000089597FB072E16F4009407D077FD09D044
:104650000E943B2307FC05D03EF4909581959F4F27
:104660000895709561957F4F0895EE0FFF1F059097
:10467000F491E02D0994AA1BBB1B51E107C0AA1FAE
:10468000BB1FA617B70710F0A61BB70B881F991FF3
:104690005A95A9F780959095BC01CD010895F99997
:1046A000FECF92BD81BDF89A992780B50895A8E103
:1046B000B0E042E050E00C947223262FF999FECF2F
:1046C0001FBA92BD81BD20BD0FB6F894FA9AF99A2F
:1046D0000FBE019608950E945D23272F0C945E2340
:1046E000DC01CB01FC01F999FECF06C0F2BDE1BDB2
:1046F000F89A319600B40D9241505040B8F70895A1
:04470000F894FFCF5B
:1047040020023F08CF08AA08760842080101BA012E
:1047140028080A03140A3F4D36391806CB059505B7
:104724005C05EF04080521053A05010203040506AA
:044734000708090069
:00000001FF
